:020000040800F2
:100000000006022001020008150F0008190F000861
:10001000710F0008190F0008450F000803020008BF
:10002000030200080302000803020008FD2700087D
:10003000030200080302000803020008030200088C
:10004000030200080302000803020008030200087C
:10005000030200080302000891390008B9390008BA
:10006000E1390008093A0008313A000803020008A3
:10007000030200080302000803020008030200084C
:10008000030200080302000803020008030200083C
:10009000030200080302000803020008593A00089E
:1000A000030200080302000803020008030200081C
:1000B000413B000803020008030200080302000895
:1000C00003020008030200080302000803020008FC
:1000D00003020008030200080302000803020008EC
:1000E000BD3A0008030200080302000803020008EA
:1000F00003020008030200080302000803020008CC
:1001000003020008030200080302000803020008BB
:1001100003020008030200080302000803020008AB
:10012000030200080302000803020008030200089B
:10013000030200080302000803020008030200088B
:10014000030200080302000803020008CD2F000884
:10015000030200080302000803020008030200086B
:10016000030200080302000803020008030200085B
:10017000030200080302000803020008030200084B
:1001800003020008030200082D3B000803020008D8
:10019000030200080302000803020008030200082B
:1001A000030200080302000803020008030200081B
:1001B000030200080302000803020008030200080B
:1001C00003020008030200080302000803020008FB
:1001D00003020008030200080302000803020008EB
:1001E00003020008030200080302000803020008DB
:1001F00003020008030200080302000803020008CB
:1002000002E000F000F8FEE772B6394880F3088893
:10021000384880F3098838484EF60851CEF200017C
:10022000086040F20000CCF200004EF63471CEF2CD
:1002300000010860BFF34F8FBFF36F8F40F20000E3
:10024000C0F2F0004EF68851CEF200010860BFF314
:100250004F8FBFF36F8F4FF00000E1EE100A4EF6A4
:100260003C71CEF200010860062080F31488BFF3D1
:100270006F8F02F027FB03F021FA4FF055301F4932
:100280001B4A91423CBF41F8040BFAE71C49194A4A
:1002900091423CBF41F8040BFAE71A491A4A1B4B3A
:1002A0009A423EBF51F8040B42F8040BF8E70020D5
:1002B0001749184A91423CBF41F8040BFAE702F093
:1002C00045FB03F065FA144C144DAC4203DA54F8C4
:1002D000041B8847F9E700F041F8114C114DAC427E
:1002E00003DA54F8041B8847F9E702F02DBB00003D
:1002F0000006022000220220000000080000022068
:1003000000060220583F0008002202205C22022042
:10031000602202205C300220000200080002000877
:1003200000020008000200082DE9F04F2DED108AB0
:10033000C1F80CD0D0F80CD0BDEC108ABDE8F08F1D
:10034000002383F311882846A047002001F080FE97
:10035000FEE701F001FE00DFFEE7000038B500F027
:10036000DBFC40B1174B6FF07F01002259720E2168
:100370001A729972DA7202F003FA044602F038FA3D
:100380000546D0B9104B9C4219D001339C4241F232
:10039000883412BF054600240125002002F0FAF936
:1003A0000DB100F05BF800F05DFD00F0F9FB2046B8
:1003B00000F0F4F800F052F8F9E70024EDE7044605
:1003C000EBE700BF00220220010007B008B500F0F3
:1003D000B3FBA0F120035842584108BD054B07B5B7
:1003E0001B88022101A8ADF8043000F0C3FB03B064
:1003F0005DF804FBD43B000810B5202383F311887B
:100400001248C3680BB101F0BFFE0023104A4FF43D
:100410007A710E4801F066FE002383F311880D4CBB
:10042000236813B12368013B2360636813B16368D9
:10043000013B6360084B1B7833B9636823B9022022
:1004400000F080FC3223636010BD00BF60220220F8
:10045000F90300087C23022074220220454B464900
:100460002DE9F04153F8042F013201D1BDE8F081AC
:100470008B42F7D1414C424B22689A4278D9414B8A
:100480009B6803F1006303F5C0339A4270D20020E9
:1004900000F0A2FB02203C4B187000F049FC3B4BE3
:1004A0001A6C00221A64196E1A66196E596C5A6415
:1004B000596E5A66596E596941F0800159615969FE
:1004C00021F0800159615969196941F000511961A0
:1004D000196921F0005119611B6972B62C4B2D4925
:1004E0000B601D682468BFF34F8FBFF36F8F2A4BDB
:1004F000C3F88420BFF34F8F5A6922F480325A61C7
:10050000BFF34F8FD3F8802043F6E07EC2F3C906D5
:10051000C2F34E32B707520102EA0E08384631469E
:10052000013948EA000C00F14040B1F1FF3FC3F847
:1005300074C2F5D1203A12F1200FEDD1BFF34F8FE5
:10054000BFF36F8FBFF34F8FBFF36F8F5A6922F4E2
:1005500000325A610022C3F85022BFF34F8FBFF31D
:100560006F8F202383F31188AD4685F308882047D9
:10057000BDE8F081FC7F01081C80010804800108AF
:10058000FF7F01080022022074220220003802406E
:100590000080010808ED00E000ED00E02DE9F04FDB
:1005A00099B0B94D2022FF21009010A8AC6800F04E
:1005B000FBFBB64A01951378A3B90121B448117029
:1005C000C360202383F31188C3680BB101F0DCFD05
:1005D0000023B04A4FF47A71AD4801F083FD002347
:1005E00083F31188009BAC4A03B113600026AB4B28
:1005F000009DB2463746B1461E70566002930120F8
:1006000000F096FB002D00F02582A34B1B68002B09
:1006100040F0208219B0BDE8F08F0220FFF7D6FE2F
:10062000002840F01082009B02210BA8002E08BF7A
:100630001D469B4B1B88ADF82C3000F09BFADEE783
:100640004FF47A7000F078FAB0F10008EBDB02208A
:10065000FFF7BCFE0028E6D008F1FF38B8F1040F20
:1006600000F2F381DFE808F0031E2124270018A818
:100670000523042140F8343D00F07CFA01234FF0BB
:10068000000903FA08F848EA0A0A5FFA8AFA00F051
:10069000DFFB27B10AF00B030B2B08BF0025FFF788
:1006A0009DFEACE704217848E6E704217D48E3E7B6
:1006B00004217D48E0E74FF01C09484609F1040990
:1006C00000F08CFA04210B900BA800F053FAB9F15A
:1006D0002C0FF2D1D2E7002FA5D00AF00B030B2B81
:1006E000A1D10220FFF772FE804600289BD0012096
:1006F0006A4E00F071FA00270220307000F018FBFB
:100700005FFA87FB584600F077FA054688B15846ED
:10071000013700F081FA0028F2D146460025634BEC
:1007200002210BA847461B88ADF82C3000F022FAB6
:1007300065E701232C460220337000F0EFFA019B9D
:100740009B689C4206D2204600F048FA0130E4D172
:100750000434F4E70024029B464647461C702546B5
:100760004D4B5C6093E7002F3FF45DAF0AF00B0345
:100770000B2B7FF458AF0220029B187000F0D8FAC0
:10078000322000F0D9F9B0F1000BFFF64CAF1BF0AE
:1007900003087FF448AF019B04EB0B0299688A427F
:1007A0003FF641AFBBF5807F3FF63DAF404AD845AD
:1007B00003920FDA4FF47A7000F0BEF904900499B6
:1007C0000029FFF630AF0499039A08F8021008F1E7
:1007D0000108ECE7C820FFF7F9FD804600283FF448
:1007E00022AF1F2C11D8C4F1200710AB24F0030056
:1007F0002F495F45184428BF5F463A4600F0ACFADF
:100800003A46FF212A4800F0CFFA4FEAAB032849C5
:100810002046DAB2039300F0CFFA074600283FF4EF
:100820007EAF039B04EB830431E70220FFF7CEFD8C
:1008300000283FF4F8AE00F015FA00283FF4F3AEBC
:100840004FF000084346019A9268904532D2B8F1C1
:100850001F0F12D8109A01320FD028F0030218A9E6
:100860000A4452F8202C0B92184604220BA908F1D6
:10087000040800F091FB0346E5E74046039300F0CF
:10088000ADF9039B0B90EFE70022022078230220B2
:1008900060220220F90300087C2302207422022037
:1008A000D63B00080422022008220220D83B000880
:1008B0007822022018A8042140F84C3D00F05AF993
:1008C000E5E618A80023642140F8343D00F048F91B
:1008D00000287FF4A8AE0220FFF778FD00283FF43F
:1008E000A2AE0B9800F0AAF918AB43F8480D04210A
:1008F0001846E3E718A80023642140F8343D00F0CF
:100900002FF900287FF48FAE0220FFF75FFD00284B
:100910003FF489AE0B9800F09FF918AB43F8440DF3
:10092000E5E70220FFF752FD00283FF47CAE00F01F
:10093000A9F918AB43F8400DD9E70220FFF746FDAF
:1009400000283FF470AE0BA9142000F0A1F98046F6
:1009500018A8042140F83C8D00F00CF941460BA882
:10096000ACE7322000F0E8F8B0F10008FFF65BAE2B
:1009700018F0030F7FF457AE019A08EB0903926851
:1009800093423FF650AE0220FFF720FD00283FF4CF
:100990004AAE28F00308C844C1453FF478AE484643
:1009A00009F1040900F01AF904210A900AA800F0DC
:1009B000E1F8F1E74FF47A70FFF708FD00283FF403
:1009C00032AE00F04FF9002842D0109B01330BD01B
:1009D000082210A9002000F0EFF9002838D02022CA
:1009E000FF2110A800F0E0F9FFF7F8FC364801F00D
:1009F00035FB0FE6002F3FF416AE0AF00B030B2B6E
:100A00007FF411AE18A80023642140F8343D00F0B3
:100A1000A7F8804600287FF406AE0220FFF7D6FC38
:100A200000283FF400AE0390FFF7D8FC41F2883075
:100A3000454601F013FB0B9800F04CFA00F008FA61
:100A4000039B1F46DBE5074621E64FF00009EAE578
:100A5000B84664E6002000F06FF80490049B002B79
:100A6000FFF6D0AD012000F059F9049B213B122B79
:100A70003FF6C5AD01A252F823F000BF1B060008E7
:100A800041060008D7060008FF050008FF0500081A
:100A9000FF05000867070008630900082B08000825
:100AA000C3080008F508000823090008FF0500082E
:100AB0003B090008FF050008B50900088F0600087B
:100AC000FF050008F5090008A08601002DE9F84F90
:100AD0004FF47A7507460E4600245543DFF85080E0
:100AE000DFF8509098F900305FFA84FA5A1C01D070
:100AF000A34210D159F82400324639460368D3F88E
:100B000020B02B46D847864205D1084B012083F8F8
:100B100000A0BDE8F88F0134022CE3D14FF4FA7045
:100B200001F09CFA0020BDE8F88F00BFC823022026
:100B30000C220220DC3B000807B5002202AB012199
:100B400003F8012D02461846FFF7C0FF20B19DF8BB
:100B5000070003B05DF804FB4FF0FF30F9E7000039
:100B60000A46042108B5FFF7B1FF80F00100C0B2CA
:100B7000404208BD074B30B41A78074B53F8224067
:100B80000A46014623682046DD69044BAC4630BC6A
:100B9000604700BFC8230220DC3B0008A08601009C
:100BA000F8B50A4C00250A4E01F0F0FC094F2080F0
:100BB00030682388834207D901F0E2FC336805449A
:100BC0000133BD423360F3D9F8BD00BFCA23022010
:100BD00084230220FF7F010001F084BD00F100604A
:100BE00000F5C0300068704700F10060920000F529
:100BF000C03001F011BD0000054B1A68054B1B8881
:100C00009B1A834202D9104401F0BABC00207047FD
:100C100084230220CA23022038B5074D04462868E1
:100C2000204401F0B5FC28B928682044BDE83840CC
:100C300001F0C6BC38BD00BF8423022010F00303BE
:100C400008D1B0F5846F05D200F10050A0F57120F5
:100C50000068704700207047014BC058704700BFC4
:100C600020F4F01F064991F8243033B10023082204
:100C7000086A81F82430FFF7B7BF0120704700BF32
:100C800088230220014B1868704700BF002004E051
:100C90001F4BF0B51E681F4BC6F30B02360C1F88A6
:100CA0005D68BA4293F9084022D09F89BA4221D0A8
:100CB0001F8BBA4206D102220C2404FB02335D686A
:100CC00093F90840B6F5805F16D041F201039E42C9
:100CD00008BF5A24421E013D0B460A44934215D2D6
:100CE00015F9016F581C4EB1034600F8016CF5E789
:100CF0000022E1E70122DFE74124EBE72C258242D5
:100D00001D7001D9981C5C70401AF0BD1846FBE7B5
:100D1000002004E01022022000207047022803D1A6
:100D20004FF08062014B9A61704700BF000C024097
:100D3000022803D14FF48062014B9A61704700BFD3
:100D4000000C0240022804D1024A536983F48063F4
:100D500053617047000C0240002310B5934203D04A
:100D6000CC5CC4540133F9E710BD000030B5441E1B
:100D700014F9010F0B4658B193F900500131854227
:100D800006D11AB993F90020801A30BD013AEFE775
:100D9000002AF7D1104630BD02460346981A13F9CF
:100DA000011B0029FAD1704702440346934202D046
:100DB00003F8011BFAE770472DE9F047234C05467D
:100DC0008846174694F8243083BB2E46DFF87C9083
:100DD000C7B394F824302BB92022FF21484626625D
:100DE000FFF7E2FF94F824004146C0F1080504EB48
:100DF0008000BD4228BF3D465FFA85FAAD00A7EBF3
:100E00000A072A462E44FFF7A7FF94F82430A84487
:100E1000FFB29A445FFA8AFABAF1080F84F824A064
:100E2000D6D1FFF71FFF0028D2D108E0266A06EBD3
:100E30008306B042CAD0FFF715FF0028C5D10020B5
:100E4000BDE8F0870120BDE8F08700BF88230220BD
:100E5000024B1A78024B1A70704700BFC823022059
:100E60000C22022038B5154C154D204600F004FC2C
:100E70002946204600F02CFC2D681248EA6ED2F874
:100E8000043843F00203C2F8043801F0E7F80E49D1
:100E9000284600F02BFDEA6E0C48D2F804380C49C5
:100EA000A04223F00203C2F804384FF4E1330B6090
:100EB00003D0BDE8384000F03DBB38BD70280220AB
:100EC000F43C000840420F001C3D00084C24022066
:100ED000B023022038B50B4B05461A780A4B53F85D
:100EE00022400A4B9C420CD0094B00211822184684
:100EF000FFF75AFF056001462046BDE8384000F084
:100F000019BB38BDC8230220DC3B00087028022032
:100F1000B0230220FEE7000000B59BB0EFF309818B
:100F200068226846FFF718FFEFF30583044B9A6BBE
:100F3000DA6A9A6A9A6A9A6A9A6A9A6A9B6AFEE76F
:100F400000ED00E000B59BB0EFF309816822684630
:100F5000FFF702FFEFF30583044B9A6B9A6A9A6AD4
:100F60009A6A9A6A9A6A9B6AFEE700BF00ED00E0FF
:100F700000B59BB0EFF3098168226846FFF7ECFEED
:100F8000EFF30583034B5A6B9A6A9A6A9A6A9A6AD4
:100F90009B6AFEE700ED00E030B50A44074D914240
:100FA0000BD011F8013B09245840013CF7D040F325
:100FB00000032B4083EA5000F7E730BD2083B8EDF3
:100FC000002304491A465A50C81808334260802B3F
:100FD000F9D17047CC2302200268436811430160B5
:100FE00003B1184770470000024A136843F0C0037A
:100FF000136070470078004013B50E4C204600F097
:101000008DFA04F11400009400234FF480720A4911
:1010100000F04EF90094094B4FF48072084904F136
:10102000380000F0C7F9074BE365074B236602B0B1
:1010300010BD00BF4C240220B8240220E90F000894
:10104000B82502200078004080F93703224B0029A0
:1010500008BF1946037C012B30B50CD11F4B9842B9
:1010600009D11F4B1A6C42F080421A641A6E42F08A
:1010700080421A661B6E0A68036EC46D03EB52034E
:101080008166B3FBF2F34A68150442BF23F00705FB
:1010900003F0070343EA4503E3608B6843F0400332
:1010A0006360CB68510543F00103A36042F496737B
:1010B00043F0010323604FF0FF33236205D512F0A4
:1010C000102205D0B2F1805F04D080F8643030BDCA
:1010D0007F23FAE73F23F8E7103C00084C24022066
:1010E000003802402DE9F047C66D05463768F469BF
:1010F000200734621AD014F0080F0CBF00218021A1
:10110000E20748BF41F02001A3074FF0200348BF8A
:1011100041F04001600748BF41F4807183F31188BA
:10112000281DFFF759FF002383F31188E2050AD534
:10113000202383F311884FF40071281DFFF74CFF23
:10114000002383F311884FF020094FF0000A14F0B8
:10115000200831D13B0616D54FF0200905F1380A99
:10116000200610D589F31188504600F057F9002861
:101170002FDA0821281DFFF72FFF27F080033360A7
:10118000002383F3118879060DD562060BD5202341
:1011900083F31188EA6C2B6D9A4201D12B6CEBB969
:1011A000002383F31188E30620D5AA6E1369EBB1FF
:1011B0005069BDE8F047184789F31188736A2846DB
:1011C00095F86410194000F0C3F98AF31188F469A6
:1011D000BDE7B06288F31188F469C1E727F04007E2
:1011E0001021281DFFF7F8FE3760D9E7BDE8F0872A
:1011F000F8B51546826804460B46AA4200D28568B7
:10120000A1692669761AB54207D218462A46FFF721
:10121000A3FDA3692B44A3610DE011D9AF1B324696
:101220001846FFF799FD3A46E1683044FFF794FD10
:10123000E2683A44A261A36828465B1BA360F8BD3C
:1012400018462A46FFF788FDE368E4E7836893427F
:101250002DE9F04104460F46154600D285686069C5
:101260002669361AB54207D22A463946FFF774FD79
:1012700063692B4463610EE013D9A5EB060832467F
:101280003946FFF769FD4246B919E068FFF764FD8A
:10129000E26842446261A36828465B1BA360BDE824
:1012A000F0812A463946FFF757FDE368E2E7000080
:1012B00010B50A440024C361029B00604060846052
:1012C000C160816141610261036210BD08B582693C
:1012D0004369934201D1826882B982680132826097
:1012E0005A1C42611970426903699A4201D3C3686A
:1012F0004361002100F0CEFE002008BD4FF0FF301A
:1013000008BD000070B5202304460E4683F3118803
:10131000A568A5B1A368A269013BA360531CA361A2
:1013200015782269934224BFE368A361E3690BB196
:1013300020469847002383F31188284670BD314624
:10134000204600F097FE0028E2DA85F3118870BD90
:101350002DE9F74F05460F4690469A46D0F81C9067
:10136000202686F311884FF0000B144664B1224604
:1013700039462846FFF73CFF034668B951462846E0
:1013800000F078FE0028F1D0002383F31188A8EB49
:10139000040003B0BDE8F08FB9F1000F03D0019055
:1013A0002846C847019B8BF31188E41A1F4486F333
:1013B0001188DBE7C160816141611144C361009B19
:1013C000006040608260016103627047F8B50446C6
:1013D0000E461746202383F31188A568A5B1A3689C
:1013E000013BA36063695A1C62611E7023696269D4
:1013F0009A4224BFE3686361E3690BB120469847D2
:10140000002080F31188F8BD3946204600F032FEF6
:101410000028E2DA85F31188F8BD0000836942698B
:101420009A4210B501D182687AB98268013282602D
:101430005A1C82611C7803699A4201D3C368836194
:10144000002100F027FE204610BD4FF0FF3010BDF8
:101450002DE9F74F05460F4690469A46D0F81C9066
:10146000202686F311884FF0000B144664B1224603
:1014700039462846FFF7EAFE034668B95146284632
:1014800000F0F8FD0028F1D0002383F31188A8EBC9
:10149000040003B0BDE8F08FB9F1000F03D0019054
:1014A0002846C847019B8BF31188E41A1F4486F332
:1014B0001188DBE7026843681143016003B11847F4
:1014C000704700001430FFF743BF00004FF0FF33B8
:1014D0001430FFF73DBF00003830FFF7B9BF000000
:1014E0004FF0FF333830FFF7B3BF00001430FFF781
:1014F00009BF00004FF0FF311430FFF703BF0000B9
:101500003830FFF763BF00004FF0FF323830FFF78D
:101510005DBF000000207047FFF76EBD044B036005
:10152000002343608360C36001230374704700BFDE
:10153000283C000810B52023044683F31188FFF7E8
:1015400085FD02232374002383F3118810BD00005E
:1015500038B5C36904460D461BB904210844FFF79A
:10156000A9FF294604F11400FFF7B0FE002806DAAF
:10157000201D4FF48061BDE83840FFF79BBF38BDA8
:10158000026843681143016003B1184770470000C7
:1015900013B5446BD4F894341A681178042915D122
:1015A000217C022912D11979012312898B4013421F
:1015B0000CD101A904F14C0001F084FFD4F894444B
:1015C0000246019B2179206800F0E0F902B010BDCD
:1015D000143001F007BF00004FF0FF33143001F06A
:1015E00001BF00004C3001F0D9BF00004FF0FF33C5
:1015F0004C3001F0D3BF0000143001F0D5BE000024
:101600004FF0FF31143001F0CFBE00004C3001F03C
:10161000A5BF00004FF0FF324C3001F09FBF00002B
:10162000D0F8942438B5136805461978042901D0F8
:10163000012038BD017C0229FAD1127901205C8990
:1016400090400440F4D105F1140001F067FE024619
:101650000028EDD0D5F894544FF480732868697948
:1016600000F082F9204638BD406BFFF7D9BF00007B
:1016700000207047704700007FB5124B01250226FD
:10168000044603600023057400F184024360294688
:101690008360C3600C4B0290143001934FF480734D
:1016A000009601F017FE094B04F5237229460193B9
:1016B00004F14C004FF480730294009601F0DEFEBA
:1016C00004B070BD503C0008691600089115000870
:1016D0000B68202282F311880A7903EB82021062E0
:1016E0004A790D3243F822008A7912B103EB820362
:1016F00018620223C0F894140374002383F3118842
:101700007047000038B5037F044613B190F8543099
:10171000ABB90125201D0221FFF732FF04F11400AF
:1017200025776FF0010100F0C1FC84F8545004F1FA
:101730004C006FF00101BDE8384000F0B7BC38BD87
:1017400010B5012104460430FFF71AFF0023237768
:1017500084F8543010BD000038B50446002514301C
:1017600001F0D0FD04F14C00257701F09FFE201D13
:1017700084F854500121FFF703FF2046BDE83840AC
:10178000FFF74EBF90F85C3003F06003202B19D1B7
:1017900090F85D20212A0AD0222A4FF000030ED0B3
:1017A000202A0FD1084A02650722426504E0064B51
:1017B00003650723436500238365012070470365A4
:1017C0004365F9E70020704734220220D0F89434B2
:1017D00037B51A680446117804291AD1017C022908
:1017E00017D11979012312898B40134211D100F1CD
:1017F0004C05284601F01AFF58B101A9284601F00E
:1018000061FED4F894440246019B2179206800F0DF
:10181000BDF803B030BD000000EB8103F7B51C6AD2
:1018200005460E46F4B1202383F3118805EB8607A5
:10183000201D08214C34FFF7A3FEFB685B691B6881
:1018400013B1204601F04CFE01A9204601F03AFEFA
:10185000024648B1019B3146284600F097F8002324
:1018600083F3118803B0F0BDFB685A691268002A3F
:10187000F5D01B8A013B1340F1D105F15C02EAE788
:101880000D3138B550F82140DCB1202383F31188A5
:10189000D4F894241368527903EB8203DB689B69C4
:1018A0005D6845B104216018FFF76AFE294604F11E
:1018B000140001F03DFD2046FFF7B2FE002383F344
:1018C000118838BD7047000001F0D2B8012300F143
:1018D000240200F1380103700023436042F8043B06
:1018E0008A421361FAD103814381704738B50446B7
:1018F000202383F3118800254160C560056145619F
:101900008561C561056201F0C3F80223237085F388
:10191000118838BD70B500EB8103054650690E464D
:101920001446DA6018B110220021FFF73DFAA069D1
:1019300018B110220021FFF737FA31462846BDE8DA
:10194000704001F06FB90000028902F001020281CB
:10195000428902F0010242810022026142618261F9
:10196000C261026201F0F2B9F0B4012500EB81041A
:1019700047898D40E4683D43A46945812360002385
:10198000A2606360F0BC01F00DBA0000F0B4012564
:1019900000EB810407898D40E4683D43646905815B
:1019A00023600023A2606360F0BC01F087BA0000EE
:1019B00070B50223002504460370A0F8645080F837
:1019C000665080F8675005814581C56005614561B5
:1019D0008561C561056280F84C5001F0BFF863680D
:1019E0001B6823B129462046BDE87040184770BDEA
:1019F000037880F868300523037043681B6810B5CE
:101A000004460BB10421984700232381638110BD54
:101A1000436890F868201B6802700BB105211847D5
:101A20007047000090F84C3070B5044613B10023A5
:101A300080F84C3004F15C02204601F0A9F963689B
:101A40009B6863BB94F85C5015F0600615D194F860
:101A50005D3005F07F0545EA032540F202339D42E3
:101A600000F00E815BD8022D00F0DC803FD8002D05
:101A700000F08780012D00F0CF800021204601F08A
:101A8000F5FB0021204601F0E7FB63681B6813B1FA
:101A9000062120469847062384F84C3070BD204626
:101AA00098470028CED094F8632094F8623043EA37
:101AB0000223626D934238BF636594F95C30656DB3
:101AC000002B4FF0200380F2FD80002D00F0EC8011
:101AD000092284F84C2083F311880021636D226D64
:101AE0002046FFF753FF002383F3118870BDB5F53F
:101AF000817F00F0B180B5F5407F49D0B5F5807F9A
:101B0000BBD194F85E30012BB7D1B4F8643023F028
:101B10000203A4F8643026656665A665C3E740F253
:101B200001639D421ED8B5F5C06F3BD2B5F5A06FDD
:101B3000A3D1B4F85C30B3F5A06F0ED194F85E3049
:101B4000204684F8663001F061F863681B6813B1C1
:101B500001212046984703232370002323656365F2
:101B6000A365A0E7B5F5106F32D040F602439D4261
:101B700052D0B5F5006F80D104F1670323650123CE
:101B800024E004F16403A5652365022363658AE705
:101B900094F85E30012B7FF470AFB4F8643043F0FA
:101BA0000203B6E794F861202046616894F860303B
:101BB0004D6843EA022394F85F1094F85E20A8472A
:101BC00000283FF45AAF4368236503686365A4E7C0
:101BD0002378042B10D1202383F311882046FFF7AC
:101BE000B3FE86F311886368032184F867601B687D
:101BF00021700BB12046984794F85E30002BACD092
:101C000084F867300423237063681B68002BA4D01A
:101C1000022120469847A0E7374B236502236365DE
:101C200000239DE794F86010204611F0800F01F02A
:101C30000F010ED001F09EF8012806D002287FF493
:101C40001CAF2E4B6065236567E72D4B65652365EB
:101C500063E701F081F8EFE794F85E30002B7FF442
:101C60000CAF94F8603013F00F013FF476AF1A0612
:101C7000204602D501F00EFB6FE701F001FB6CE797
:101C800094F85E30002B7FF4F8AE94F8603013F0D7
:101C90000F013FF462AF1B06204602D501F0E6FAC1
:101CA0005BE701F0D9FA58E7142284F84C2083F35B
:101CB00011882B462A4629462046FFF755FE85F314
:101CC000118870BD5DB1152284F84C2083F3118812
:101CD0000021636D226D2046FFF746FE03E70B22CD
:101CE00084F84C2083F311882B462A462946204647
:101CF000FFF74CFEE3E700BF803C0008783C00089B
:101D00007C3C000838B590F84C300446152B29D897
:101D1000DFE803F03E28282828283E28280B293908
:101D200028282828282828283E3E90F8631090F874
:101D30006220436D42EA01229A4214D9C268128A93
:101D4000B3FBF2F502FB15356DB9202383F311883F
:101D50002B462A462946FFF719FE85F311880A23E8
:101D600084F84C3038BD142384F84C30202383F39E
:101D70001188002320461A461946FFF7F5FD002377
:101D800083F3118838BD836D03B198470023E7E7DB
:101D9000002101F06BFA0021204601F05DFA636832
:101DA0001B6813B10621204698470623D8E7000098
:101DB00090F84C20152A38B5044622D801239340C8
:101DC00040F6416213421DD113F480150FD19B02DE
:101DD00017D50B2380F84C30202383F311882B4632
:101DE0002A462946FFF7D2FD85F3118838BDC3681E
:101DF0009B695B682BB9836D03B19847002384F816
:101E00004C3038BD002101F031FA0021204601F0AC
:101E100023FA63681B6813B10621204698470623FE
:101E2000EDE70000024B00221B605B609A60704788
:101E3000B8260220002382680374054B1B6899684A
:101E40009142FBD25A68036042601060586070474C
:101E5000B826022008B5202383F31188037C032BC6
:101E600005D0042B0DD02BB983F3118808BD43692D
:101E700000221A604FF0FF334361FFF7DBFF0023BE
:101E8000F2E790E80C001A6002685360F2E7000085
:101E9000002382680374054B1B6899689142FBD844
:101EA0005A6803604260106058607047B82602208C
:101EB000054B196908741868026853601A60186144
:101EC00001230374FEF730BAB82602204B1C30B54C
:101ED000054687B00A4C10D0236901A8094A00F0D2
:101EE00001F92846FFF7E4FF049B13B101A800F0B5
:101EF0004BF92369586907B030BDFFF7D9FFF8E700
:101F0000B8260220551E000838B50C4D0446416124
:101F10002B6981689A68914203D8BDE83840FFF781
:101F200089BF1846FFF7B4FF01232C6101462374D3
:101F30002046BDE83840FEF7F7B900BFB8260220BA
:101F4000044B1A681B6990689B68984294BF0020F4
:101F500001207047B826022010B5084C236820697C
:101F60001A6854602260012223611A74FFF790FFFF
:101F700001462069BDE81040FEF7D6B9B826022018
:101F8000FEE7000010B50C4CFFF74CFF00F09CF88A
:101F900080220A49204600F021F8012344F8180C59
:101FA000037400F03BFC002383F3118862B60448FD
:101FB000BDE8104000F034B8E0260220843C000860
:101FC0008C3C000800F01AB9034B59685A68521A41
:101FD0009042FBD8704700BF001000E082600222F0
:101FE00002740022427470478368A3F17C0243F8B4
:101FF0000C2C026943F83C2C426943F8382C074A00
:1020000043F81C2CC268A3F1180043F8102C0222DC
:1020100003F8082C002203F8072C7047410300083E
:1020200010B5202383F31188FFF7DEFF002104465B
:10203000FFF76AFF002383F31188204610BD0000DC
:10204000024B1B6958610F20FFF732BFB8260220F0
:10205000202383F31188FFF7F3BF000008B5014682
:10206000202383F311880820FFF730FF002383F338
:10207000118808BD49B1064B42681B6918605A6057
:10208000136043600420FFF721BF4FF0FF3070471B
:10209000B82602200368984206D01A680260506091
:1020A00018465961FFF7C6BE7047000038B50446B0
:1020B0000D462068844200D138BD036823605C600F
:1020C0004561FFF7B7FEF4E7054B03F114025A61CF
:1020D0009A614FF0FF32DA6100221A62704700BF46
:1020E000B8260220F8B5274F0D4603610446C260AA
:1020F0003E4601F0CFFA3B46022D294653F8142FF5
:1021000038BF02219A421D460AD1386208447C61D8
:10211000BC6122606260A160BDE8F84001F0A8BA2D
:10212000D7F820E0A0EB0E035F181FD300279068BC
:10213000834217D8376AAA421F44376201D0C01AB7
:10214000906073699A68914219D85A6823606260F6
:1021500014605C60A1609868411A99604FF0FF3389
:10216000F361F8BD97601B1A1268E0E793689F421D
:1021700003D20EEB070001F089FA3946E1E7891A2C
:102180001B68DFE7B826022038B51B4B01685A6987
:102190001D46904203F114020CD0446821600021D6
:1021A000036893425C60C16025D09A6881680A44E4
:1021B0009A6038BD59614A6000215B69C1609342F1
:1021C00003D1BDE8384001F05BBA9A6881680A44DF
:1021D0009A602C6A01F05EFA6A69001B926882427A
:1021E00009D9111A012998BF821C286ABDE8384014
:1021F000104401F04BBA38BDB82602202DE9F84F43
:10220000204C0027656904F11406B84601F042FA33
:10221000236AA0EB030AAB6853451DD84FF0200991
:10222000236AAA68D5F80CB013442362AB68AAEB02
:10223000030A2B68B3425E606361EF6001D101F075
:102240001FFA88F311882869D84789F311886569CE
:10225000AB689A45E4D2D9E76369B34210D02062F3
:102260009A68A2EB0A029A60226AAB68821A9B1AE9
:10227000022B2CBFC0180230BDE8F84F01F006BA9F
:10228000BDE8F88FB826022000207047FEE7000066
:10229000704700004FF0FF3070470000022906D061
:1022A000032906D00129064818BF002070470548B9
:1022B0007047032A9ABF044800EBC2000020704711
:1022C000783D00082C3D00083C22022070B59AB0F1
:1022D00006460846144601AD294600F095F8284602
:1022E000FEF75AFDC0B2431C5B0086E8180023705D
:1022F0000323023404F8013C00231946DAB2023405
:10230000904201D81AB070BDEA5C013304F8011C98
:1023100004F8022CF2E7000008B5202383F31188AB
:102320000348FFF753FA002383F3118808BD00BF69
:102330007028022010B50446052916D8DFE801F000
:1023400016150316161D202383F311880E4A01214A
:10235000FFF7E0FA20460D4A0221FFF7DBFA0C48AE
:10236000FFF7FAF9002383F3118810BD202383F3CC
:1023700011880748FFF7C6F9F4E7202383F3118893
:102380000348FFF7DDF9EDE7AC3C0008D03C00085E
:102390007028022038B50C4D0C4C2A460C4904F12B
:1023A0000800FFF793FF05F1CA0204F11000094984
:1023B000FFF78CFF05F5CA7204F118000649BDE865
:1023C0003840FFF783BF00BF382D02203C22022097
:1023D000FC3C0008063D0008113D000870B50446AD
:1023E00008460D46FEF7D8FCC6B2204601340378F5
:1023F0000BB9184670BD32462946FEF7B7FC0028D7
:10240000F3D1012070BD00002DE9F84F05460C46C0
:10241000FEF7C2FC2C49C6B22846FFF7DFFF08B121
:102420000536F6B229492846FFF7D8FF08B110361D
:10243000F6B2632E0DD8DFF89080DFF89090244F2D
:10244000DFF894A0DFF894B02E7846B92670BDE886
:10245000F88F29462046BDE8F84F01F0B3BB252E82
:102460002ED1072241462846FEF780FC70B9DBF8E2
:10247000003007350C3444F80C3CDBF8043044F8E9
:10248000083CDBF8083044F8043CDDE70822494604
:102490002846FEF76BFC98B9A21C0E4B13F8011FDF
:1024A000023209095345C95D02F8041C197801F08C
:1024B0000F01C95D02F8031CF0D118340835C3E7D9
:1024C000267001350134BFE7983D0008113D000832
:1024D000AD3D00081FF4F01F2BF4F01FA03D0008D5
:1024E000BFF34F8F024AD368DB03FCD4704700BFB1
:1024F000003C024008B5074B1B7853B9FFF7F0FFCB
:10250000054B1A69002A04DA044A5A6002F188323B
:102510005A6008BD962F0220003C02402301674507
:1025200008B5054B1B7833B9FFF7DAFF034A136987
:1025300043F00043136108BD962F0220003C024087
:102540000B2870B513D80B4A0B4C137863B94FF0B6
:1025500000610A4E44F8231056F8235001330C2B27
:102560002944F7D10123137054F8200070BD0020D6
:1025700070BD00BFC82F0220982F0220C03D000868
:10258000014B53F820007047C03D00080C207047F5
:102590000B2810B5044601D9002010BDFFF7D0FF6D
:1025A000064B53F824301844C21A0BB9012010BD51
:1025B00012680132F0D1043BF6E700BFC03D0008CD
:1025C0000B2810B5044621D8FFF78AFFFFF792FFCA
:1025D0000F4AF323D360C300DBB243F4007343F02C
:1025E00002031361136943F480331361FFF778FF2B
:1025F000FFF7A6FF074B53F8241000F0DBF8FFF7B6
:102600008FFF2046BDE81040FFF7C2BF002010BD7D
:10261000003C0240C03D00082DE9F84312F00103E0
:1026200015463FD18218B2F1026F3BD22B4B1B688B
:1026300013F0010336D0FFF75DFF294CF32340F27E
:102640000127E360FFF74CFF032D01D9830712D068
:102650000F46401A224C40F20118EB1BC6190B44DE
:10266000012B236924D823F001032361FFF758FFCE
:102670000120BDE8F883236923F4407323612369B3
:102680003B43236151F8046B0660BFF34F8FFFF7A4
:1026900027FF03689E4208D0236923F001032361CA
:1026A000FFF73EFF0020BDE8F883043D0430CBE790
:1026B00023F44073B9462361236943EA0803236185
:1026C00037F8023B3380BFF34F8FFFF709FF36889F
:1026D000B6B2B9F80030B342BFD0DDE700380240EF
:1026E000003C0240084908B50B7828B153B9FFF700
:1026F00001FF01230B7008BD23B10870BDE808403D
:10270000FFF70EBF08BD00BF962F02200244043918
:10271000064BD2B210B5904200D110BD441C00B29D
:1027200053F8200041F8040FE0B2F4E750280040CD
:10273000104B30B51C6F240407D41C6F44F4007494
:102740001C671C6F44F400441C670B4C02440439A2
:102750002368D2B243F480732360084B904200D1C7
:1027600030BD441C51F8045F00B243F82050E0B281
:10277000F4E700BF003802400070004050280040DD
:1027800007B5012201A90020FFF7C0FF019803B09F
:102790005DF804FB13B50446FFF7F2FFA04206D034
:1027A00002A90122002041F8044DFFF7C1FF02B049
:1027B00010BD00000144BFF34F8F064B884204D385
:1027C000BFF34F8FBFF36F8F7047C3F85C022030A9
:1027D000F4E700BF00ED00E0034B1B689B0042BF25
:1027E0000122024B1A70704774380240C92F022030
:1027F000014B1878704700BFC92F0220EFF30983FF
:10280000054968334A6822F001024A6083F3098867
:10281000002383F31188704730EF00E0202080F31D
:10282000118862B60D4B0E4AD96821F4E0610904A3
:10283000090C0A430B49DA60CA6842F08072CA6028
:10284000094A0A49C2F8B01F116841F0010111603C
:102850001022DA7783F82200704700BF00ED00E015
:102860000003FA05F0ED00E0001000E055CEACC525
:1028700010B5202383F311880E4B5B6813F40063BB
:1028800014D0F1EE103AEFF309844FF08073683CF6
:10289000E361094BDB68236684F30988FFF750FB8B
:1028A00010B1064BA36110BD054BFBE783F3118804
:1028B00010BD00BF00ED00E030EF00E05303000862
:1028C00056030008F0B5BFF34F8FBFF36F8F1D4B5A
:1028D0000021C3F85012BFF34F8FBFF36F8F5A69B7
:1028E00042F400325A61BFF34F8FBFF36F8FC3F8CA
:1028F0008410BFF34F8FD3F8802043F6E076C2F305
:10290000C904C2F34E32A507520102EA060E284658
:1029100021464EEA0007013900F14040C3F86072D9
:102920004F1CF6D1203A12F1200FEED1BFF34F8F9A
:102930005A6942F480325A61BFF34F8FBFF36F8FF1
:10294000F0BD00BF00ED00E0FEE70000084A094BC3
:1029500009498B4204D3094A0021934205D37047A9
:1029600052F8040F43F8040BF3E743F8041BF4E7B1
:10297000B03F00085C3002205C3002205C30022056
:10298000036F002170B5C46E4FF0FF359E684A0199
:10299000A318D3F80009002805DAD3F8000940F09D
:1029A0008040C3F80009D3F8000B002805DAD3F8FB
:1029B000000B40F08040C3F8000B0131A3188E4299
:1029C000C3F80859C3F8085BE1D24FF00113C4F80B
:1029D0001C3870BD890141F02001016103699B062B
:1029E000FCD41220FFF7F0BA204B03EB80022DE954
:1029F000F047D2F80CE0461CDD6EDEF8142005EB43
:102A00000636D2F800C005EB4018516861450BD37B
:102A10000123D5F8342803FA00F022EA0000C5F8B3
:102A200034081846BDE8F087ACEB0103BEF810404F
:102A3000A34228BF2346D8F81849A4B2B3EB840FA9
:102A400010D894681F46A4F1040959F804AF042F64
:102A5000C6F800A001D9043FF7E71C440B4494607A
:102A60005360D2E70020BDE8F08700BFCC2F0220E2
:102A700010B5054C2046FEF729FF4FF0A043E36652
:102A8000024B236710BD00BFCC2F0220143E00086C
:102A90000378012B70B5054650D12A4BC46E98427D
:102AA0001BD1294B0E2143205A6B42F080025A63FE
:102AB0005A6D42F080025A655A6D5A6942F080029E
:102AC0005A615A6922F080025A615B6900F0ECFB9E
:102AD0001E4BE3601E4BC4F800380023EE6EC4F8B2
:102AE000003EC02323604FF40413A3633369002B1B
:102AF000FCDA01230C203361FFF766FA3369DB0748
:102B0000FCD41220FFF760FA3369002BFCDA0026B0
:102B10002846A660FFF734FF6B68C4F81068DB68CE
:102B2000C4F81468C4F81C684BB90A4BA3614FF091
:102B3000FF336361A36843F00103A36070BD064BDC
:102B4000F4E700BFCC2F02200038024040140040C0
:102B500003002002003C30C0083C30C0F8B5C46E11
:102B6000054600214FF000662046FFF733FF296F2E
:102B700000234FF001128F684FF0FF30C4F8343853
:102B8000C4F81C2804EB431201339F42C2F80069C9
:102B9000C2F8006BC2F80809C2F8080BF2D20B6841
:102BA000EA6E6B67636210231361166916F01006F4
:102BB000FBD11220FFF708FAD4F8003823F4FE63A3
:102BC000C4F80038A36943F4402343F01003A36121
:102BD0000923C4F81038C4F814380A4BEB604FF0DE
:102BE000C043C4F8103B084BC4F8003BC4F810695C
:102BF000C4F800396B6F03F1100243F480136A6765
:102C0000A362F8BDF03D000840800010C26E90F84D
:102C10006610D2F8003823F4FE6343EA0113C2F8C9
:102C2000003870472DE9F0410EB20D4600EB8608E2
:102C3000D8F80C100F6807F00303022B50D0032BB9
:102C400050D03D4A3D4F012B18BF1746C46E4FEA86
:102C5000451E002205F1100C04EB0E03C3F8102BE7
:102C60008A69002A40D04A8A05F158033A435B0139
:102C7000E2500123D4F81C2803FA0CF31343C4F8E0
:102C80001C38A64400234A69CEF8103905F13F03E9
:102C9000002A39D00A8A04EB8303898B9208012920
:102CA00088BF4A43416F561841EA024229464667A7
:102CB00020465A60FFF78EFED8F80C301B8A43EA94
:102CC00085531F4305F148035B01E7500123D4F806
:102CD0001C2803FA05F51543C4F81C58BDE8F0811B
:102CE000174FB3E7174FB1E704EB4613D3F8002BA8
:102CF00022F40042C3F8002B0123D4F81C2803FA65
:102D00000CF322EA0303BAE704EB83030E4A04EB55
:102D1000461629465A602046FFF75CFED6F8003971
:102D2000012223F4004302FA05F5C6F80039D4F86D
:102D30001C3823EA0505CFE700800010008004104E
:102D40000080081000800C1000040002026F12685E
:102D50004267FFF715BE00005831C36E49015B584A
:102D600013F4004004D013F4001F14BF012002200C
:102D7000704700004831C36E49015B5813F40040AE
:102D800004D013F4001F14BF01200220704700007C
:102D900000EB8101CB68196A0B6813604B685360C4
:102DA0007047000000EB810330B5DD68AA69136845
:102DB000D36019B9402B84BF402313606B8A146819
:102DC000C26E1C4402EB4110013C09B2B4FBF3F4A7
:102DD0006343033323F0030343EAC44343F0C04394
:102DE000C0F8103B2B6803F00303012B0ED1D2F87F
:102DF000083802EB411013F4807FD0F8003B14BF79
:102E000043F0805343F00053C0F8003B02EB411203
:102E1000D2F8003B43F00443C2F8003B30BD000051
:102E20002DE9F041244D0446EE6E06EB4013D3F835
:102E3000087B3807C3F8087B0AD5D6F81438190779
:102E400006D505EB840321462846DB685B68984776
:102E5000FA072FD5D6F81438DB072BD505EB8403FA
:102E6000D968CCB98B69488A5E68B6FBF0F200FB82
:102E700012628AB91868DA6890420DD2121A83E891
:102E80001400202383F311880B482146FFF78AFFA3
:102E900084F31188BDE8F081012303FA04F26B8901
:102EA00023EA02036B81CB6823B121460248BDE8C7
:102EB000F0411847BDE8F081CC2F022000EB8103E0
:102EC0004A0170B5DD68C36E6C692668E66056BB62
:102ED0001A444FF40020C2F810092A6802F00302D5
:102EE000012A0AB20ED1D3F8080803EB421410F4F9
:102EF000807FD4F8000914BF40F0805040F00050AB
:102F0000C4F8000903EB4212D2F8000940F0044073
:102F1000C2F800090122D3F8340802FA01F1014392
:102F2000C3F8341870BD19B9402E84BF402020600A
:102F300020681A442E8A841940F00050013CB4FBEA
:102F4000F6F440EAC440C6E7F8B504461E48C56E2C
:102F500005EB4413D3F80869F107C3F8086917D5DE
:102F6000D5F81038DA0713D500EB8403D9684B691C
:102F70001F68DA68974218D2D21B00271A605F6078
:102F8000202383F311882146FFF798FF87F31188E8
:102F9000330617D50123D5F83428A340134211D0A6
:102FA0002046BDE8F840FFF71FBD012303FA04F2F5
:102FB000038923EA020303818B68002BE8D02146B2
:102FC0009847E5E7F8BD00BFCC2F0220A1482DE9C6
:102FD000F84FC56E04466E69AB691E4016F4805FFB
:102FE0006E6105D0FEF7E4FCBDE8F84FFFF740BC8A
:102FF000002E12DAD5F8003E9B0705D0D5F8003E2A
:1030000023F00303C5F8003ED5F80438914823F0B7
:103010000103C5F80438FEF7FBFC370505D58D48DC
:10302000FFF7AEFC8B48FEF7E3FCB0040CD5D5F8F7
:10303000083813F0060FEB6823F470530CBF43F409
:10304000105343F4A053EB60310704D56368DB6889
:103050000BB180489847F2026FD4B3020CD5D4F874
:103060006C8000274FF00109DFF8E8A1236FF9B267
:103070009B688B4280F09C80F70619D5E16E0A6A46
:10308000C2F30A1702F00F0302F4F012B2F5802F18
:1030900000F0B580B2F5402F0AD104EB830301F5AF
:1030A0008051DB68186A00231A469F4240F09C80DA
:1030B0003303D5F818481DD5E70302D50020FFF7E4
:1030C000AFFEA50302D50120FFF7AAFE600302D5DB
:1030D0000220FFF7A5FE210302D50320FFF7A0FE83
:1030E000E20202D50420FFF79BFEA30202D50520D1
:1030F000FFF796FE77037FF577AFE60702D500204E
:10310000FFF722FFA50702D50120FFF71DFF60078B
:1031100002D50220FFF718FF210702D50320FFF791
:1031200013FFE20602D50420FFF70EFFA3067FF58A
:103130005BAF0520FFF708FF56E7D4F86C80002747
:103140004FF00109DFF80CA1236F5FFA87FB9B6842
:103150005B4582D308EB4B13D3F8002902F44022DD
:10316000B2F5802F22D1D3F80029002A1EDAD3F835
:10317000002942F09042C3F80029D3F80029002A20
:10318000FBDB5946E06EFFF725FC228909FA0BF3B9
:1031900022EA0303238104EB8B03DB689B6813B1F2
:1031A0005946504698475846FFF71EFC0137CBE773
:1031B00008EB4112D2F8003B03F44023B3F5802F13
:1031C00010D1D2F8003B002B0CDA628909FA01F326
:1031D00022EA0303638104EB8103DB68DB680BB144
:1031E00050469847013741E79C0700D10A68072BF2
:1031F00003F101039EBF0270120A013055E702334A
:1032000001F5805104EB8302526890690268D0F89E
:1032100008C04068A2EB000E0022104697420AD177
:1032200004EB830463689B699A683A449A605A681D
:1032300017445F603CE712F0030F00D10868964521
:1032400002F1010282BF8CF80000000A0CF1010CAF
:10325000E4E700BFCC2F0220C36E03EB4111D1F88D
:10326000003B43F40013C1F8003B7047C36E03EB0F
:103270004111D1F8003943F40013C1F80039704707
:10328000C36E03EB4111D1F8003B23F40013C1F8E6
:10329000003B7047C36E03EB4111D1F8003923F4B2
:1032A0000013C1F80039704700F1604300F01F02BD
:1032B0000901400903F56143C9B2800083F8001396
:1032C000012300F16040934000F56140C0F8803177
:1032D0000360704730B50433039C0172002104FB86
:1032E0000325C361049B00600363059B4060C160CC
:1032F000426102618561046242628162C16243632C
:1033000030BD00000022416AC260416101616FF07E
:1033100001018262C262FEF7C9BE00000369426910
:10332000934203D1C2680AB100207047181D70474C
:10333000036919600021C2680132C260C269134486
:1033400082699342036124BF436A0361FEF7A2BE10
:1033500038B504460D46E3683BB162690020131D91
:103360001268A3621344E36238BD237A33B9294655
:103370002046FEF77FFE0028EDDA38BD6FF0010031
:10338000FBE70000C368C269013BC36043691344A3
:1033900082699342436124BF436A4361002383628D
:1033A000036B03B11847704770B52023044683F3BD
:1033B0001188866A3EB9FFF7CBFF054618B186F340
:1033C0001188284670BDA36AE26A13F8015B934234
:1033D000A36202D32046FFF7D5FF002383F31188B1
:1033E000EFE700002DE9F84F04460E469046994657
:1033F000202787F311880025AA46D4F828B0BBF10E
:10340000000F09D149462046FFF7A2FF20B18BF3F8
:1034100011882846BDE8F88FA16AA8EB050BE36A7E
:103420005B1A9B4528BF9B46BBF1400F1BD9334617
:1034300001F1400251F8040B914243F8040BF9D119
:10344000A36A403640354033A362A26AE36A9A42D7
:1034500002D32046FFF796FF8AF311884545D8D25C
:1034600087F31188C9E730465A46FDF775FCA36A11
:103470005E445D445B44A362E7E7000010B5029C34
:1034800004330172C36103FB0421002300608362E3
:10349000C362039B40600363049BC460426102619A
:1034A000816104624262436310BD0000026A6FF0F2
:1034B0000101C260426A4261026100228262C2620C
:1034C000FEF7F4BD436902699A4203D1C2680AB1AA
:1034D00000207047184650F8043B0B60704700000E
:1034E000C3680021C2690133C36043691344826920
:1034F0009342436124BF436A4361FEF7CBBD0000A2
:1035000038B504460D46E3683BB1236900201A1D17
:10351000A262E2691344E36238BD237A33B92946D3
:103520002046FEF7A7FD0028EDDA38BD6FF0010058
:10353000FBE7000003691960C268013AC260C26912
:10354000134482699342036124BF436A03610023E9
:103550008362036B03B118477047000070B52023E6
:1035600004460E4683F31188856A35B91146FFF784
:10357000C7FF10B185F3118870BDA36A1E70A36ADE
:10358000E26A01339342A36204D3E169204604391D
:10359000FFF7D0FF002080F3118870BD2DE9F84FB0
:1035A00004460D4691469A464FF0200888F311884C
:1035B0000026B346A76A4FB951462046FFF7A0FF41
:1035C00020B187F311883046BDE8F88FA06AA9EBD7
:1035D0000603E76A3F1A9F4228BF1F46402F1BD9A8
:1035E00005F1400355F8042B9D4240F8042BF9D116
:1035F000A36A40364033A362A26AE36A9A4204D3C4
:10360000E16920460439FFF795FF8BF311884E4599
:10361000D9D288F31188CDE729463A46FDF79CFBBD
:10362000A36A3D443E443B44A362E5E70269436923
:103630009A4203D1C3681BB9184670470023FBE7C1
:10364000836A002BF8D0043B9B1AF5D01360C36843
:10365000013BC360C3691A4483699A42026124BF73
:10366000436A0361002383620123E5E700F09EB80B
:103670004FF08043002258631A610222DA607047DB
:1036800000224FF08043DA60704700004FF0804323
:10369000586370474FF08043586A70474B684360E7
:1036A0008B688360CB68C3600B6943614B690362BD
:1036B0008B6943620B6803607047000008B5274BB5
:1036C00040F2FF7126481A690A431A611A6922F406
:1036D000FF6222F007021A611A691A6B0A431A6321
:1036E0001A6D0A431A651F4A1B6D1146FFF7D6FF74
:1036F0001D4802F11C01FFF7D1FF1C4802F13801FF
:10370000FFF7CCFF1A4802F15401FFF7C7FF194831
:1037100002F17001FFF7C2FF174802F18C01FFF7B9
:10372000BDFF164802F1A801FFF7B8FF144802F1E7
:10373000C401FFF7B3FF134802F1E001FFF7AEFF4A
:10374000114802F1FC01FFF7A9FF104802F58C7146
:10375000FFF7A4FFBDE8084000F09EB80038024023
:1037600000000240203E0008000402400008024021
:10377000000C0240001002400014024000180240F9
:10378000001C0240002002400024024000280240A9
:1037900008B500F005FAFEF7F5FBFFF71DF8BDE8E8
:1037A0000840FEF7F7BD0000704700000F4B1A6C91
:1037B00042F001021A641A6E42F001021A660C4AC3
:1037C0001B6E936843F0010393604FF080436B22BC
:1037D0009A624FF0FF32DA6200229A615A63DA602D
:1037E0005A6001225A611A60704700BF00380240D7
:1037F000002004E04FF0804208B51369D1680B4007
:10380000D9B29B076FEA0101116107D5202383F329
:103810001188FEF7D7FB002383F3118808BD000051
:103820001B4B4FF0FF3000211A696FEA42526FEADA
:1038300052521A611A69C2F30A021A611A695A6964
:1038400058615A6959615A691A6A62F080521A625B
:103850001A6A02F080521A621A6A5A6A58625A6ADE
:1038600059625A6A0B4A106840F480701060186FF1
:1038700000F44070B0F5007F03D04FF4803018673B
:103880001967536823F40073536000F061B900BFF7
:103890000038024000700040374B4FF44041374A37
:1038A0001A64374A11601A6842F001021A601A68F5
:1038B0009207FCD59A6822F003029A602E4B1946B3
:1038C0009A6812F00C02FBD1186800F0F900186039
:1038D0009A601A6842F480321A600B689B03FCD528
:1038E0004B6F43F001034B67234B5A6F9007FCD596
:1038F000244A5A601A6842F080721A60204B1A46B5
:1039000059684904FCD5196841F48031196053683D
:10391000D803FCD5136843F400331360184A536886
:103920009903FCD5144B1A689201FCD5164A9A608B
:1039300040F20112C3F88C200022C3F8902040F21C
:103940000732124B1A601A6802F00F02072AFAD1E6
:10395000094B9A6842F002029A609A6802F00C02DF
:10396000082AFAD15A6C42F480425A645A6E42F4E0
:1039700080425A665B6E70470038024000040010B7
:1039800000700040086C400900948838003C0240F8
:10399000074A08B5536903F00103536123B1054A8F
:1039A00013680BB150689847BDE80840FEF760BF48
:1039B000003C0140CC230220074A08B5536903F0BC
:1039C0000203536123B1054A93680BB1D06898474D
:1039D000BDE80840FEF74CBF003C0140CC2302206C
:1039E000074A08B5536903F00403536123B1054A3C
:1039F00013690BB150699847BDE80840FEF738BF1E
:103A0000003C0140CC230220074A08B5536903F06B
:103A10000803536123B1054A93690BB1D0699847F4
:103A2000BDE80840FEF724BF003C0140CC23022043
:103A3000074A08B5536903F01003536123B1054ADF
:103A4000136A0BB1506A9847BDE80840FEF710BFF3
:103A5000003C0140CC230220164B10B55C6904F4F5
:103A600078725A61A30604D5134A936A0BB1D06ADF
:103A70009847600604D5104A136B0BB1506B9847FA
:103A8000210604D50C4A936B0BB1D06B9847E20525
:103A900004D5094A136C0BB1506C9847A30504D5A3
:103AA000054A936C0BB1D06C9847BDE81040FEF707
:103AB000DFBE00BF003C0140CC230220194B10B5F3
:103AC0005C6904F47C425A61620504D5164A136DA0
:103AD0000BB1506D9847230504D5134A936D0BB174
:103AE000D06D9847E00404D50F4A136E0BB1506EA9
:103AF0009847A10404D50C4A936E0BB1D06E984739
:103B0000620404D5084A136F0BB1506F9847230421
:103B100004D5054A936F0BB1D06F9847BDE81040AC
:103B2000FEF7A6BE003C0140CC23022008B50348A6
:103B3000FDF7D8FABDE80840FEF79ABE4C240220F3
:103B400008B5FFF757FEBDE80840FEF791BE00003C
:103B5000062108B50846FFF7A7FB06210720FFF757
:103B6000A3FB06210820FFF79FFB06210920FFF792
:103B70009BFB06210A20FFF797FB06211720FFF782
:103B800093FB06212820FFF78FFB07211C20FFF75E
:103B90008BFB0C215220BDE80840FFF785BB0000DD
:103BA00008B5FFF73DFEFDF70BFAFDF7B5FCFDF795
:103BB0008BFEFDF75FFDFFF7F7FDBDE80840FFF75F
:103BC00055BD0000034611F8012B03F8012B002A14
:103BD000F9D1704712101213121100007028022040
:103BE0004C24022053544D3332463F3F3F3F3F3F2A
:103BF0000053544D333246375B347C355D78005387
:103C0000544D333246375B367C375D780000000018
:103C1000009600000000000000000000000000000E
:103C2000000000000000000000000000E114000897
:103C3000CD14000809150008F51400080115000846
:103C4000ED140008D9140008C51400081515000863
:103C500000000000ED150008D91500081516000831
:103C6000011600080D160008F9150008E5150008F2
:103C7000D1150008711600080000000001000000C6
:103C8000000000006D61696E00000000A43C0008A7
:103C9000F82602207028022001000000811F000881
:103CA0000000000069646C65000000000200000074
:103CB00000000000191800088118000840004000AA
:103CC000082D0220182D0220020000000000000034
:103CD0000300000000000000C518000800000000FC
:103CE00010000000282D022000000000010000004C
:103CF00000000000CC2F0220010102004172647517
:103D000050696C6F740025424F415244252D424C3E
:103D1000002553455249414C250000003523000839
:103D20009D220008851700081923000843000000A1
:103D3000343D000809024300020100C032090400BA
:103D40000001020201000524001001052401000108
:103D5000042402020524060001070582030800FF6F
:103D600009040100020A00000007050102400000EA
:103D7000070581024000000012000000803D00089D
:103D80001201100102000040091241570002010215
:103D9000030100000403090425424F415244250059
:103DA0004D6174656B463736352D534500303132E1
:103DB00033343536373839414243444546000000F4
:103DC00000800000008000000080000000800000F3
:103DD00000000200000004000000040000000400D5
:103DE00000000400000004000000040000000400C3
:103DF00000000000251A0008051D0008B11D00087C
:103E00004000400044300220443002200100000005
:103E10005430022080000000400100000500000036
:103E20000000802A00000000AAAAAAAA0000000040
:103E3000FFFF00000000000000A00A0000000001D9
:103E400000000000AAAAAAAA00000001FFFF0000CB
:103E50000000000000000000000100000000000061
:103E6000AAAAAAAA00010000FFFF000000000000AB
:103E7000000000000040100000000000AAAAAAAA4A
:103E800000400000FFFB00000000000000000000F8
:103E90000080420000000000AAAAAAAA0040410037
:103EA000FFFF00000000008008000000000000008C
:103EB00000000000AAAAAAAA00000000FFFF00005C
:103EC00000000000000000000000000000000000F2
:103ED000AAAAAAAA00000000FFFF0000000000003C
:103EE000000000000000000000000000AAAAAAAA2A
:103EF00000000000FFFF00000000000000000000C4
:103F00000000000000000000AAAAAAAA0000000009
:103F1000FFFF0000000000000000000000000000A3
:103F20000000000000000000000000000000000091
:103F30000000000000000000000000000000000081
:103F40000000000000000000000000000000000071
:103F500000000000000000008F00000000000000D2
:103F600000801E00FF00000000000000E43B00088D
:103F70003F00000049040000F13B00083F00000042
:103F800051040000FF3B00083F00000000960000C5
:103F90000000080004000000943D0008000000003C
:103FA0000000000000000000000000000000000011
:043FB000000000000D
:00000001FF
